:020000040000FA
:0408000063EF09F0A9
:1008100003B283EF05F0F2B4A1EF05F09EB0A9EFAB
:1008200005F09EB2B1EF05F0F2A81AEF04F0F2B2B3
:1008300032EF04F09EB61FEF04F012EF09F09E961F
:1008400000011450000A06E000011450010A06E0FD
:1008500012EF09F079EC20F012EF09F071EC22F0C0
:1008600012EF09F0CD90F2929EA03CEF04F001014E
:10087000533F3CEF04F0542BAEC1B2F1AFC1B3F122
:10088000B0C1B4F1B1C1B5F1AAC1AEF1ABC1AFF124
:10089000ACC1B0F1ADC1B1F1A6C1AAF1A7C1ABF134
:1008A000A8C1ACF1A9C1ADF1A2C1A6F1A3C1A7F144
:1008B000A4C1A8F1A5C1A9F19EC1A2F19FC1A3F154
:1008C000A0C1A4F1A1C1A5F19AC19EF19BC19FF164
:1008D0009CC1A0F19DC1A1F196C19AF197C19BF174
:1008E00098C19CF199C19DF1CECF96F1CFCF97F1F0
:1008F00053C198F154C199F1CF6ACE6A0101536B8B
:10090000546B9E90CD800FBC0F8E0FBA8BEF04F00E
:100910000F8A12EF09F00F8C0FBEC7EF04F096C1DB
:100920009AF197C19BF198C19CF199C19DF19AC12F
:100930009EF19BC19FF19CC1A0F19DC1A1F19EC1FF
:10094000A2F19FC1A3F1A0C1A4F1A1C1A5F1A2C1CF
:10095000A6F1A3C1A7F1A4C1A8F1A5C1A9F1A6C19F
:10096000AAF1A7C1ABF1A8C1ACF1A9C1ADF1AAC16F
:10097000AEF1ABC1AFF1ACC1B0F1ADC1B1F1AEC13F
:10098000B2F1AFC1B3F1B0C1B4F1B1C1B5F1010180
:100990005E6B5F6B606B616B96515E2797515F2357
:1009A00098516023995161239A515E279B515F238F
:1009B0009C5160239D5161239E515E279F515F236F
:1009C000A0516023A1516123A2515E27A3515F234F
:1009D000A4516023A5516123A6515E27A7515F232F
:1009E000A8516023A9516123AA515E27AB515F230F
:1009F000AC516023AD516123AE515E27AF515F23EF
:100A0000B0516023B1516123B2515E27B3515F23CE
:100A1000B4516023B5516123D89001016133603333
:100A20005F335E33D8900101613360335F335E33EF
:100A3000D8900101613360335F335E3300C10CF144
:100A400001C10DF102C10EF103C10FF104C110F19A
:100A500005C111F106C112F107C113F108C114F16A
:100A600009C115F10AC116F10BC117F134C135F1F5
:100A700011B846EF05F00101620E046F010E056F1B
:100A8000000E066F000E076F4FEF05F00101A70E75
:100A9000046F020E056F000E066F000E076F5EC139
:100AA00000F15FC101F160C102F161C103F110EC1D
:100AB0001FF003BF04D019BE02D019A0108C11A0E2
:100AC00067EF05F010BA67EF05F00F80108A0CC1D0
:100AD00000F10DC101F10EC102F10FC103F110C10E
:100AE00004F111C105F112C106F113C107F114C1DE
:100AF00008F115C109F116C10AF117C10BF135C191
:100B000034F112EF09F00392ABB2AB98AB8803015A
:100B100003EE00F080517F0BE92604C0EFFF802B2D
:100B20008151805D700BD8A48B8200008051815D63
:100B3000700BD8A48B9281518019D8B4079012EF12
:100B400009F0F2940101453F12EF09F0462B12EF34
:100B500009F09E900101533F12EF09F0542B12EF60
:100B600009F09E9211B820EF07F08BB4BFEF05F0AB
:100B700010ACBFEF05F08B84109CC0EF05F08B9498
:100B8000C3CF55F1C4CF56F1C28207B42AEF06F0A5
:100B900047C14BF148C14CF149C14DF14AC14EF139
:100BA0005EC162F15FC163F160C164F161C165F171
:100BB00096C1B6F197C1B7F198C1B8F199C1B9F131
:100BC0009AC1BAF19BC1BBF19CC1BCF19DC1BDF101
:100BD0009EC1BEF19FC1BFF1A0C1C0F1A1C1C1F1D1
:100BE000A2C1C2F1A3C1C3F1A4C1C4F1A5C1C5F1A1
:100BF000A6C1C6F1A7C1C7F1A8C1C8F1A9C1C9F171
:100C0000AAC1CAF1ABC1CBF1ACC1CCF1ADC1CDF140
:100C1000AEC1CEF1AFC1CFF1B0C1D0F1B1C1D1F110
:100C2000B2C1D2F1B3C1D3F1B4C1D4F1B5C1D5F1E0
:100C3000010155515B2756515C23E86A5D230E2E56
:100C40002AEF06F05CC157F15DC158F15B6B5C6B3C
:100C50005D6B078E0201002F12EF09F03C0E006F52
:100C60001A50E00BE00AE866128818BE02D018B4E9
:100C7000108E00C10CF101C10DF102C10EF103C1D2
:100C80000FF104C110F105C111F106C112F107C144
:100C900013F108C114F109C115F10AC116F10BC114
:100CA00017F134C135F101018A675EEF06F08B67F9
:100CB0005EEF06F08C675EEF06F08D6762EF06F080
:100CC00092EF06F08EC100F18FC101F190C102F1E7
:100CD00091C103F10101010E046F000E056F000EBA
:100CE000066F000E076F10EC1FF000C18EF101C1FE
:100CF0008FF102C190F103C191F1006787EF06F017
:100D0000016787EF06F0026787EF06F0036792EF4F
:100D100006F08AC18EF18BC18FF18CC190F18DC12B
:100D200091F10F80D57ED5BE6DD0D6CF47F1D7CF0C
:100D300048F145C149F1E86AE8CF4AF119BE02D04D
:100D400019A0108C109047C100F148C101F149C1B0
:100D500002F14AC103F101010A0E046F000E056F92
:100D6000000E066F000E076F10EC1FF003AF10802F
:100D7000010154A7C8EF06F00F9A0F9C0F9E0101C6
:100D8000000E5E6F600E5F6F3D0E606F080E616F4C
:100D9000010147BFD8EF06F04867D8EF06F0496772
:100DA000D8EF06F04A67D8EF06F0F288FDEF06F0BC
:100DB000F2985E6B5F6B606B616B966B976B986B79
:100DC000996B9A6B9B6B9C6B9D6B9E6B9F6BA06BE7
:100DD000A16BA26BA36BA46BA56BA66BA76BA86B97
:100DE000A96BAA6BAB6BAC6BAD6BAE6BAF6BB06B47
:100DF000B16BB26BB36BB46BB56BD76AD66A0101DA
:100E0000456B466B0CC100F10DC101F10EC102F141
:100E10000FC103F110C104F111C105F112C106F1B6
:100E200013C107F114C108F115C109F116C10AF186
:100E300017C10BF135C134F112EF09F012EF09F0CF
:100E40000201002F79EF08F0D59ED6CF47F1D7CF1A
:100E500048F145C149F1E86AE8CF4AF1D76AD66A54
:100E60000101456B466BD58E1A50E00BE00AE8662F
:100E7000128818BE02D018B4108E17AE1C8C00C198
:100E80000CF101C10DF102C10EF103C10FF104C15A
:100E900010F105C111F106C112F107C113F108C12A
:100EA00014F109C115F10AC116F10BC117F134C1D2
:100EB00035F10FA0109A11B869EF07F00101620E29
:100EC000046F010E056F000E066F000E076F72EFC4
:100ED00007F00101A70E046F020E056F000E066FEA
:100EE000000E076F47C100F148C101F149C102F18D
:100EF0004AC103F110EC1FF003BF85EF07F019BEE4
:100F000002D019A0108C11B00F800CC100F10DC1DE
:100F100001F10EC102F10FC103F110C104F111C1C1
:100F200005F112C106F113C107F114C108F115C191
:100F300009F116C10AF117C10BF135C134F10201F3
:100F40003C0E006F00C10CF101C10DF102C10EF1A8
:100F500003C10FF104C110F105C111F106C112F175
:100F600007C113F108C114F109C115F10AC116F145
:100F70000BC117F134C135F101018A67C7EF07F0E2
:100F80008B67C7EF07F08C67C7EF07F08D67CBEF74
:100F900007F0FBEF07F08EC100F18FC101F190C1A6
:100FA00002F191C103F10101010E046F000E056F02
:100FB000000E066F000E076F10EC1FF000C18EF1DF
:100FC00001C18FF102C190F103C191F10067F0EF0F
:100FD00007F00167F0EF07F00267F0EF07F0036733
:100FE000FBEF07F08AC18EF18BC18FF18CC190F1BC
:100FF0008DC191F10F80109047C100F148C101F1FE
:1010000049C102F14AC103F101010A0E046F000E49
:10101000056F000E066F000E076F10EC1FF003AF98
:101020001080010154A721EF08F00F9A0F9C0F9E2A
:101030000101000E5E6F600E5F6F3D0E606F080E67
:10104000616F47C100F148C101F149C102F14AC1D4
:1010500003F10101140E046F050E056F000E066FFB
:10106000000E076F10EC1FF003AF3AEF08F0F288A4
:101070005FEF08F0F2985E6B5F6B606B616B966B75
:10108000976B986B996B9A6B9B6B9C6B9D6B9E6B34
:101090009F6BA06BA16BA26BA36BA46BA56BA66BE4
:1010A000A76BA86BA96BAA6BAB6BAC6BAD6BAE6B94
:1010B000AF6BB06BB16BB26BB36BB46BB56B0CC198
:1010C00000F10DC101F10EC102F10FC103F110C118
:1010D00004F111C105F112C106F113C107F114C1E8
:1010E00008F115C109F116C10AF117C10BF135C19B
:1010F00034F130EC23F01D661ED01CAE11D01C9EC6
:101100001D8E18AE07D0146A040E156E166A79EC9F
:1011100020F011D0146A156A166A79EC20F00BD011
:101120001CAC09D01C9C1D8C010E146E156A166A2D
:1011300071EC22F000D08BB4A5EF08F010ACA5EF55
:1011400008F08B84109CA6EF08F08B94C3CF55F168
:10115000C4CF56F1C28207B410EF09F047C14BF17A
:1011600048C14CF149C14DF14AC14EF15EC162F135
:101170005FC163F160C164F161C165F196C1B6F10F
:1011800097C1B7F198C1B8F199C1B9F19AC1BAF153
:101190009BC1BBF19CC1BCF19DC1BDF19EC1BEF123
:1011A0009FC1BFF1A0C1C0F1A1C1C1F1A2C1C2F1F3
:1011B000A3C1C3F1A4C1C4F1A5C1C5F1A6C1C6F1C3
:1011C000A7C1C7F1A8C1C8F1A9C1C9F1AAC1CAF193
:1011D000ABC1CBF1ACC1CCF1ADC1CDF1AEC1CEF163
:1011E000AFC1CFF1B0C1D0F1B1C1D1F1B2C1D2F133
:1011F000B3C1D3F1B4C1D4F1B5C1D5F10101555199
:101200005B2756515C23E86A5D230E2E10EF09F030
:101210005CC157F15DC158F15B6B5C6B5D6B078E18
:1012200012EF09F002C0E0FF005001C0D8FF10002B
:10123000A6B218EF09F00CC0A9FF0BC0A8FFA69E2C
:10124000A69CA684F29E550EA76EAA0EA76EA68235
:10125000F28EA694A6B22AEF09F00C2A1200A96E0B
:10126000A69EA69CA680A8500C2A120004012C0E53
:10127000826F3BEC0BF00BEC20F00C502FEC09F0E4
:10128000E8CF00F10C502FEC09F0E8CF01F101AFED
:101290004FEF09F00101FF0E026FFF0E036FAEEC7E
:1012A0001FF029675BEF09F00401200E826F3BEC11
:1012B0000BF060EF09F004012D0E826F3BEC0BF098
:1012C000B8EC1DF01200306A076A0F6A106A116AE2
:1012D000126A136A0F010E0EC16E860EC06E030EE7
:1012E000C26E0F01896A110E926E080E8A6EF10E9F
:1012F000936E8B6A980E946EF18EFC0E2FEC09F0B3
:10130000E8CF0BF00BA011800BA211820BA411846B
:101310000BA81188C90E2FEC09F0E8CF17F0CA0E00
:101320002FEC09F0E8CF18F0CB0E2FEC09F0E8CF46
:1013300019F0CC0E2FEC09F0E8CF1AF0CD0E2FECFF
:1013400009F0E8CF2FF01C6A1D6A0E6A01015B6B81
:101350005C6B5D6B576B586BF29A0101476B486B86
:10136000496B4A6B4B6B4C6B4D6B4E6B4F6B506BC1
:10137000516B526B456B466BD76AD66A0F01280ECC
:10138000D56EF28A9D90B00ECD6E01015E6B5F6BE3
:10139000606B616B626B636B646B656B666B676BD9
:1013A000686B696B536B546BCF6ACE6A0F9A0F9C54
:1013B0000F9E9D80760ECA6E9D8202013C0E006FCC
:1013C000CC6A160E2FEC09F0E8CF00F1170E2FECC7
:1013D00009F0E8CF01F1180E2FEC09F0E8CF02F187
:1013E000190E2FEC09F0E8CF03F1010103AF13EF61
:1013F0000AF00BEC20F0160E0C6E00C10BF018EC8E
:1014000009F0170E0C6E01C10BF018EC09F0180E64
:101410000C6E02C10BF018EC09F0190E0C6E03C132
:101420000BF018EC09F000C18AF101C18BF102C187
:101430008CF103C18DF100C18EF101C18FF102C1A8
:1014400090F103C191F11A0E2FEC09F0E8CF00F1F1
:101450001B0E2FEC09F0E8CF01F11C0E2FEC09F068
:10146000E8CF02F11D0E2FEC09F0E8CF03F10101E6
:1014700003AF69EF0AF00BEC20F01A0E0C6E00C1FE
:101480000BF018EC09F01B0E0C6E01C10BF018EC00
:1014900009F01C0E0C6E02C10BF018EC09F01D0EC9
:1014A0000C6E03C10BF018EC09F01A0E2FEC09F0CA
:1014B000E8CF00F11B0E2FEC09F0E8CF01F11C0E74
:1014C0002FEC09F0E8CF02F11D0E2FEC09F0E8CF68
:1014D00003F100C192F101C193F102C194F103C182
:1014E00095F1240EAC6E900EAB6E240EAC6E080E11
:1014F000B86E000EB06E1F0EAF6E0401806B816B74
:101500000F01900EAB6E0F019D8A0301806B816B02
:10151000C26B8B92146A156A166A9D860790000149
:10152000F28EF28C07B061EF1CF00FB0FCEF15F0FB
:1015300010BEFCEF15F012B8FCEF15F0030180515E
:1015400081197F0BD8B461EF1CF013EE00F08151CC
:101550007F0BE126812BE7CFE8FFE00BD8B461EFEA
:101560001CF023EE82F0C2513F0BD926E7CFDFFFFC
:10157000C22BDF50780AD8A461EF1CF007808EC11F
:1015800000F18FC101F190C102F191C103F101019C
:10159000040E046F000E056F000E066F000E076F3D
:1015A00010EC1FF000AFDEEF0AF00101030E8E6FAA
:1015B000000E8F6F000E906F000E916F030182512D
:1015C000720AD8B4E1EF15F08251520AD8B4E1EFB3
:1015D00015F08251750AD8B4E1EF15F08251630A13
:1015E000D8B41BEF19F08251690AD8B488EF12F011
:1015F00082517A0AD8B49BEF13F08251490AD8B4C9
:1016000027EF12F08251500AD8B431EF11F0825115
:10161000700AD8B479EF11F08251540AD8B4A9EF06
:1016200011F08251740AD8B4F4EF11F08251410ADA
:10163000D8B451EF0CF082514B0AD8B44FEF0BF0F5
:1016400082516D0AD8B484EF10F082514D0AD8B49B
:101650009DEF10F08251730AD8B411EF15F082514A
:10166000530AD8B476EF15F08251590AD8B4D5EFA1
:101670000FF052EF19F0040114EE00F080517F0BCF
:10168000E12682C4E7FF802B120004010D0E826F59
:101690003BEC0BF00A0E826F3BEC0BF012000401E6
:1016A0004B0E826F3BEC0BF004012C0E826F3BEC77
:1016B0000BF081B802D02FB630D003018351430A1A
:1016C000D8B494EF0BF003018351630AD8B496EFBA
:1016D0000BF003018351520AD8B498EF0BF00301C9
:1016E0008351720AD8B49AEF0BF003018351470A71
:1016F000D8B49CEF0BF003018351670AD8B49EEF76
:101700000BF003018351540AD8B4A0EF0BF003018E
:101710008351740AD8B40FEF0CF003018351550ABA
:10172000D8B4A2EF0BF082D02F807AD02F9078D04F
:101730002F8276D02F9274D02F8472D02F9470D0B5
:101740002F866ED084C330F185C331F186C332F168
:1017500087C333F10101296B59EC20F0D0EC1FF065
:1017600000C104F101C105F102C106F103C107F195
:101770004CEC20F0200EF86EF76AF66A0900F5CFFF
:101780002CF10900F5CF2DF10900F5CF2EF109005C
:10179000F5CF2FF10900F5CF30F10900F5CF31F188
:1017A0000900F5CF32F10900F5CF33F10101296BC2
:1017B00059EC20F0D0EC1FF010EC1FF00067E8EFC0
:1017C0000BF00167E8EF0BF00267E8EF0BF003673F
:1017D00001D025D004014E0E826F3BEC0BF00401CA
:1017E0006F0E826F3BEC0BF004014D0E826F3BECF1
:1017F0000BF00401610E826F3BEC0BF00401740EE0
:10180000826F3BEC0BF00401630E826F3BEC0BF03C
:101810000401680E826F3BEC0BF050EF19F02F962D
:10182000CD0E0C6E2FC00BF018EC09F0CD0E2FEC86
:1018300009F0E8CF2FF02FB006D00401630E826FBD
:101840003BEC0BF005D00401430E826F3BEC0BF038
:101850002FB206D00401720E826F3BEC0BF005D064
:101860000401520E826F3BEC0BF02FB406D0040142
:10187000670E826F3BEC0BF005D00401470E826FC0
:101880003BEC0BF02FB606D00401740E826F3BECDC
:101890000BF005D00401540E826F3BEC0BF050EFBF
:1018A00019F00401410E826F3BEC0BF003018351F0
:1018B000310AD8B4F5EF0EF003018351320AD8B4DF
:1018C00025EF0EF003018351330AD8B4AEEF0DF0CB
:1018D00003018351340AD8B49EEF0CF00301835105
:1018E000350AD8B47BEF0CF004013F0E826F3BEC5D
:1018F0000BF050EF19F004012C0E826F3BEC0BF053
:1019000003018451300AD8B48EEF0CF003018451E6
:10191000310AD8B496EF0CF0E7EF0DF08B9004018C
:10192000300E826F3BEC0BF09CEF0CF08B800401CF
:10193000310E826F3BEC0BF050EF19F0CC0E2FEC18
:1019400009F0E8CF0BF004012C0E826F3BEC0BF09A
:1019500003018451310AD8B4C2EF0CF00301845161
:10196000300AD8B4C4EF0CF0030184514D0AD8B446
:10197000CEEF0CF003018451540AD8B4D5EF0CF02B
:10198000ECEF0CF08A8401D08A940BAE04D00BAC3F
:1019900002D00BBA21D0E00E0B1218D01F0E0B167E
:1019A0008539E844E00B0B1211D0E00E0B164CEC1D
:1019B00020F085C332F186C333F10101296B59EC64
:1019C00020F0D0EC1FF000511F0B0B12CC0E0C6E50
:1019D0000BC00BF018EC09F00401340E826F3BECE5
:1019E0000BF004012C0E826F3BEC0BF0CC0E2FECB5
:1019F00009F0E8CF1AF08AB406D00401300E826FE5
:101A00003BEC0BF005D00401310E826F3BEC0BF088
:101A100004012C0E826F3BEC0BF01A38E840070BE8
:101A2000E8CF82F40401300E82273BEC0BF0040176
:101A30002C0E826F3BEC0BF00BEC20F01A501F0BBE
:101A4000E8CF00F1AEEC1FF032C182F40401300E99
:101A500082273BEC0BF033C182F40401300E822765
:101A60003BEC0BF004012C0E826F3BEC0BF00BEC0B
:101A700020F02DC000F100AF0BD0FF0E016FFF0E64
:101A8000026FFF0E036F04012D0E826F3BEC0BF013
:101A9000AEEC1FF031C182F40401300E82273BEC22
:101AA0000BF032C182F40401300E82273BEC0BF0C4
:101AB00033C182F40401300E82273BEC0BF00401A9
:101AC0002C0E826F3BEC0BF00BEC20F02CC000F1E5
:101AD000AEEC1FF031C182F40401300E82273BECE2
:101AE0000BF032C182F40401300E82273BEC0BF084
:101AF00033C182F40401300E82273BEC0BF0040169
:101B00002C0E826F3BEC0BF00BEC20F02EC000F1A2
:101B100000AF0BD0FF0E016FFF0E026FFF0E036FC1
:101B200004012D0E826F3BEC0BF0AEEC1FF031C1C7
:101B300082F40401300E82273BEC0BF032C182F4B8
:101B40000401300E82273BEC0BF033C182F4040118
:101B5000300E82273BEC0BF050EF19F0CB0E2FEC40
:101B600009F0E8CF0BF004012C0E826F3BEC0BF078
:101B700003018451450AD8B4D2EF0DF0030184511A
:101B8000440AD8B4D5EF0DF003018451300AD8B41B
:101B9000D8EF0DF003018451310AD8B4DCEF0DF019
:101BA000E7EF0DF00B9EE1EF0DF00B8EE1EF0DF086
:101BB000FC0E0B16E1EF0DF0FC0E0B160B80E1EFA7
:101BC0000DF0CB0E0C6E0BC00BF018EC09F00401FD
:101BD000330E826F3BEC0BF004012C0E826F3BEC5A
:101BE0000BF0CB0E2FEC09F0E8CF19F019BE00EF87
:101BF0000EF00401450E826F3BEC0BF005EF0EF08A
:101C00000401440E826F3BEC0BF004012C0E826F3A
:101C10003BEC0BF00401300E826F3BEC0BF0040147
:101C20002C0E826F3BEC0BF019B01EEF0EF004018E
:101C3000300E826F3BEC0BF023EF0EF00401310EFF
:101C4000826F3BEC0BF050EF19F0CA0E2FEC09F04D
:101C5000E8CF0BF004012C0E826F3BEC0BF003017C
:101C60008451450AD8B461EF0EF003018451440A4F
:101C7000D8B464EF0EF0030184514D0AD8B46DEF6F
:101C80000EF003018451410AD8B467EF0EF003014E
:101C90008451460AD8B46AEF0EF003018451560A03
:101CA000D8B475EF0EF003018451500AD8B480EF18
:101CB0000EF003018451520AD8B483EF0EF08CEF7A
:101CC0000EF00B9E86EF0EF00B8E86EF0EF00B9C47
:101CD00086EF0EF00B8C86EF0EF0FC0E0B1685C314
:101CE000E8FF030B0B1286EF0EF0C70E0B1685C331
:101CF000E8FF070BE846E846E8460B1286EF0EF0D1
:101D00000B8486EF0EF00B9486EF0EF0CA0E0C6E6D
:101D10000BC00BF018EC09F0CA0E2FEC09F0E8CF5D
:101D200018F00401320E826F3BEC0BF004012C0E14
:101D3000826F3BEC0BF018BEA5EF0EF00401450ED0
:101D4000826F3BEC0BF0AAEF0EF00401440E826FA1
:101D50003BEC0BF004012C0E826F3BEC0BF018C037
:101D6000E8FF030BE8CF82F40401300E82273BEC3E
:101D70000BF004012C0E826F3BEC0BF018BCC8EF8B
:101D80000EF00401410E826F3BEC0BF0CDEF0EF034
:101D90000401460E826F3BEC0BF004012C0E826FA7
:101DA0003BEC0BF018C0E8FF380BE842E842E84291
:101DB000E8CF82F40401300E82273BEC0BF00401E3
:101DC0002C0E826F3BEC0BF018B4EEEF0EF004011A
:101DD000520E826F3BEC0BF0F3EF0EF00401500E4D
:101DE000826F3BEC0BF050EF19F0C90E2FEC09F0AD
:101DF000E8CF0BF004012C0E826F3BEC0BF00301DB
:101E00008451450AD8B413EF0FF003018451440AFA
:101E1000D8B416EF0FF0030184514D0AD8B419EF6E
:101E20000FF027EF0FF00B9E21EF0FF00B8E21EF3D
:101E30000FF0F80E0B1685C3E8FF070B0B1221EF0E
:101E40000FF0C90E0C6E0BC00BF018EC09F004017A
:101E5000310E826F3BEC0BF004012C0E826F3BECD9
:101E60000BF0C90E2FEC09F0E8CF17F017BE06D023
:101E70000401450E826F3BEC0BF005D00401440ECB
:101E8000826F3BEC0BF004012C0E826F3BEC0BF0ED
:101E900017C0E8FF070BE8CF82F40401300E822759
:101EA0003BEC0BF004012C0E826F3BEC0BF0078037
:101EB0000BEC20F028C0E8FF003B00430043030B7D
:101EC000AEEC1FF033C182F40401300E82273BECEC
:101ED0000BF004012C0E826F3BEC0BF00BEC20F0AE
:101EE00028C001F1019F019D29C000F10101AEEC64
:101EF0001FF02FC182F40401300E82273BEC0BF05F
:101F000030C182F40401300E82273BEC0BF031C16A
:101F100082F40401300E82273BEC0BF032C182F4D4
:101F20000401300E82273BEC0BF033C182F4040134
:101F3000300E82273BEC0BF004012C0E826F3BEC41
:101F40000BF00BEC20F02AC001F12BC000F1D8906F
:101F500001330033D890013300330101AEEC1FF0A0
:101F60002FC182F40401300E82273BEC0BF030C10C
:101F700082F40401300E82273BEC0BF031C182F475
:101F80000401300E82273BEC0BF032C182F40401D5
:101F9000300E82273BEC0BF033C182F40401300E8B
:101FA00082273BEC0BF050EF19F0FC0E2FEC09F000
:101FB000E8CF0BF003018351520AD8B40CEF10F0B4
:101FC00003018351720AD8B40FEF10F0030183515B
:101FD000500AD8B412EF10F003018351700AD8B43C
:101FE00015EF10F003018351550AD8B418EF10F023
:101FF00003018351750AD8B41BEF10F0030183511C
:10200000430AD8B424EF10F003018351630AD8B413
:1020100027EF10F030EF10F00B902AEF10F00B804C
:102020002AEF10F00B922AEF10F00B822AEF10F03B
:102030000B942AEF10F00B842AEF10F00B962AEF86
:1020400010F00B862AEF10F00B982AEF10F00B8897
:102050002AEF10F0FC0E0C6E0BC00BF018EC09F020
:102060000401590E826F3BEC0BF011901192119408
:102070001198FC0E2FEC09F0E8CF0BF00BA01180AB
:102080000BA211820BA411840BA8118811A050EF90
:1020900010F00401520E826F3BEC0BF055EF10F084
:1020A0000401720E826F3BEC0BF011A85FEF10F091
:1020B0000401430E826F3BEC0BF064EF10F004015F
:1020C000630E826F3BEC0BF011A26EEF10F0040177
:1020D000500E826F3BEC0BF073EF10F00401700EAA
:1020E000826F3BEC0BF011A47DEF10F00401550E54
:1020F000826F3BEC0BF082EF10F00401750E826FE3
:102100003BEC0BF050EF19F004016D0E826F3BECCD
:102110000BF003018351300AD8B4E1EF10F0030152
:102120008351310AD8B4F4EF10F003018351320A1D
:10213000D8B407EF11F052EF19F081B803D02FB4E3
:1021400050EF19F004014D0E826F3BEC0BF04CEC9C
:1021500020F084C331F185C332F186C333F101012C
:10216000296B59EC20F0D0EC1FF003018351300AA9
:10217000D8B4C9EF10F003018351310AD8B4D1EFBC
:1021800010F003018351320AD8B4D9EF10F052EFA6
:1021900019F0FD0E0C6E00C10BF018EC09F0E1EF28
:1021A00010F0FE0E0C6E00C10BF018EC09F0F4EF0D
:1021B00010F0FF0E0C6E00C10BF018EC09F007EFE9
:1021C00011F00401300E826F3BEC0BF004012C0E79
:1021D000826F3BEC0BF00BEC20F0FD0E2FEC09F0C6
:1021E000E8CF00F118EF11F00401310E826F3BECE3
:1021F0000BF004012C0E826F3BEC0BF00BEC20F08B
:10220000FE0E2FEC09F0E8CF00F118EF11F00401F9
:10221000320E826F3BEC0BF00BEC20F004012C0E25
:10222000826F3BEC0BF0FF0E2FEC09F0E8CF00F1D2
:10223000AEEC1FF031C182F40401300E82273BEC7A
:102240000BF032C182F40401300E82273BEC0BF01C
:1022500033C182F40401300E82273BEC0BF050EFC7
:1022600019F081B803D02FB227EF12F083C32AF1FF
:1022700084C32BF185C32CF186C32DF187C32EF1C6
:1022800088C32FF189C330F18AC331F18BC332F196
:102290008CC333F1010159EC20F0D0EC1FF0160E85
:1022A0000C6E00C10BF018EC09F0170E0C6E01C19A
:1022B0000BF018EC09F0180E0C6E02C10BF018ECC4
:1022C00009F0190E0C6E03C10BF018EC09F000C1F7
:1022D0008AF101C18BF102C18CF103C18DF100C102
:1022E0008EF101C18FF102C190F103C191F127EF8D
:1022F00012F081B803D02FB227EF12F083C32AF176
:1023000084C32BF185C32CF186C32DF187C32EF135
:1023100088C32FF189C330F18AC331F18BC332F105
:102320008CC333F1010159EC20F0D0EC1FF000C157
:102330008AF101C18BF102C18CF103C18DF100C1A1
:102340008EF101C18FF102C190F103C191F127EF2C
:1023500012F081B803D02FB227EF12F083C32AF115
:1023600084C32BF185C32CF186C32DF187C32EF1D5
:1023700088C32FF189C330F18AC331F18CC332F1A4
:102380008DC333F1010159EC20F0D0EC1FF00101B5
:10239000000E046F000E056F010E066F000E076F32
:1023A00021EC1FF01A0E0C6E00C10BF018EC09F0B6
:1023B0001B0E0C6E01C10BF018EC09F01C0E0C6E1C
:1023C00002C10BF018EC09F01D0E0C6E03C10BF0EE
:1023D00018EC09F000C192F101C193F102C194F12E
:1023E00003C195F127EF12F081B803D02FB227EF88
:1023F00012F083C32AF184C32BF185C32CF186C369
:102400002DF187C32EF188C32FF189C330F18AC320
:1024100031F18CC332F18DC333F1010159EC20F05D
:10242000D0EC1FF00101000E046F000E056F010ECD
:10243000066F000E076F21EC1FF000C192F101C181
:1024400093F102C194F103C195F127EF12F0160E3A
:102450002FEC09F0E8CF00F1170E2FEC09F0E8CFD0
:1024600001F1180E2FEC09F0E8CF02F1190E2FEC54
:1024700009F0E8CF03F1AEEC1FF071EC1DF00401A0
:10248000730E826F3BEC0BF004012C0E826F3BEC61
:102490000BF08AC100F18BC101F18CC102F18DC139
:1024A00003F1AEEC1FF071EC1DF00401730E826FAE
:1024B0003BEC0BF004012C0E826F3BEC0BF01A0E80
:1024C0002FEC09F0E8CF00F11B0E2FEC09F0E8CF5C
:1024D00001F11C0E2FEC09F0E8CF02F11D0E2FECDC
:1024E00009F0E8CF03F16DEC19F004012C0E826FB6
:1024F0003BEC0BF092C100F193C101F194C102F1E8
:1025000095C103F16DEC19F045EC0BF052EF19F0A9
:102510000401690E826F3BEC0BF004012C0E826FFC
:102520003BEC0BF00101040E006F000E016F000E7A
:10253000026F000E036FAEEC1FF02CC182F4040199
:10254000300E82273BEC0BF02DC182F40401300EDB
:1025500082273BEC0BF02EC182F40401300E82275F
:102560003BEC0BF02FC182F40401300E82273BECD0
:102570000BF030C182F40401300E82273BEC0BF0EB
:1025800031C182F40401300E82273BEC0BF032C1E2
:1025900082F40401300E82273BEC0BF033C182F44D
:1025A0000401300E82273BEC0BF004012C0E826FED
:1025B0003BEC0BF00101030E006F000E016F000EEB
:1025C000026F000E036FAEEC1FF02CC182F4040109
:1025D000300E82273BEC0BF02DC182F40401300E4B
:1025E00082273BEC0BF02EC182F40401300E8227CF
:1025F0003BEC0BF02FC182F40401300E82273BEC40
:102600000BF030C182F40401300E82273BEC0BF05A
:1026100031C182F40401300E82273BEC0BF032C151
:1026200082F40401300E82273BEC0BF033C182F4BC
:102630000401300E82273BEC0BF004012C0E826F5C
:102640003BEC0BF00101340E006F000E016F000E29
:10265000026F000E036FAEEC1FF02CC182F4040178
:10266000300E82273BEC0BF02DC182F40401300EBA
:1026700082273BEC0BF02EC182F40401300E82273E
:102680003BEC0BF02FC182F40401300E82273BECAF
:102690000BF030C182F40401300E82273BEC0BF0CA
:1026A00031C182F40401300E82273BEC0BF032C1C1
:1026B00082F40401300E82273BEC0BF033C182F42C
:1026C0000401300E82273BEC0BF004012C0E826FCC
:1026D0003BEC0BF0200EF86EF76AF66A0401090075
:1026E000F5CF82F43BEC0BF00900F5CF82F43BEC24
:1026F0000BF00900F5CF82F43BEC0BF00900F5CFAD
:1027000082F43BEC0BF00900F5CF82F43BEC0BF0CC
:102710000900F5CF82F43BEC0BF00900F5CF82F411
:102720003BEC0BF00900F5CF82F43BEC0BF045ECF1
:102730000BF052EF19F081B803D02FB0EBEF13F08C
:102740008351630AD8A450EF19F08451610AD8A4C8
:1027500050EF19F085516C0AD8A450EF19F086514A
:10276000410A42E08651440A1BE08651420AD8B42D
:1027700007EF14F08651350AD8B4DCEF1AF0865111
:10278000360AD8B431EF1BF08651370AD8B49AEF25
:102790001BF08651380AD8B4F8EF1BF050EF19F04F
:1027A0000798079A04017A0E826F3BEC0BF0040144
:1027B000780E826F3BEC0BF00401640E826F3BECF1
:1027C0000BF081A8EBEF13F00401550E826F3BEC88
:1027D0000BF0F0EF13F004014C0E826F3BEC0BF0AA
:1027E00045EC0BF052EF19F00788079A04017A0EB6
:1027F000826F3BEC0BF00401410E826F3BEC0BF05F
:102800000401610E826F3BEC0BF0E1EF13F00798CF
:10281000078A04017A0E826F3BEC0BF00401420E32
:10282000826F3BEC0BF00401610E826F3BEC0BF00E
:10283000E1EF13F00101666725EF14F0676725EFFC
:1028400014F0686725EF14F0696715D04F6730EF13
:1028500014F0506730EF14F0516730EF14F0526706
:102860000AD00101000E006F000E016F000E026F12
:10287000000E036F120011B80AD00101620E046F3E
:10288000010E056F000E066F000E076F09D00101E3
:10289000A70E046F020E056F000E066F000E076F85
:1028A00066C100F167C101F168C102F169C103F1BC
:1028B00010EC1FF003BFCDEF14F0119A119C010131
:1028C000000E046FA80E056F550E066F020E076FFF
:1028D00066C100F167C101F168C102F169C103F18C
:1028E00066C186F167C187F168C188F169C189F164
:1028F00010EC1FF003BF0BD00101000E866FA80E75
:10290000876F550E886F020E896F118A119C0E0E0B
:102910002FEC09F0E8CF18F10F0E2FEC09F0E8CFFB
:1029200019F1100E2FEC09F0E8CF1AF1110E2FEC6F
:1029300009F0E8CF1BF159EC1EF086C104F187C104
:1029400005F188C106F189C107F110EC1FF007827B
:102950001DEC1EF059EC1EF007921DEC1EF086C116
:1029600000F187C101F188C102F189C103F1079229
:102970001DEC1EF0CC0E046FE00E056F870E066F87
:10298000050E076F10EC1FF000C118F101C119F11D
:1029900002C11AF103C11BF13BD0119C119A010134
:1029A000800E006F1A0E016F060E026F000E036F8D
:1029B0004FC104F150C105F151C106F152C107F1F7
:1029C00010EC1FF003AF05D00BEC20F0118C119A26
:1029D00012000E0E2FEC09F0E8CF18F10F0E2FECBD
:1029E00009F0E8CF19F1100E2FEC09F0E8CF1AF139
:1029F000110E2FEC09F0E8CF1BF14FC100F150C1CF
:102A000001F151C102F152C103F107821DEC1EF028
:102A100018C100F119C101F11AC102F11BC103F182
:102A200012000401730E826F3BEC0BF004012C0EBC
:102A3000826F3BEC0BF0078462C166F163C167F102
:102A400064C168F165C169F14BC14FF14CC150F1EE
:102A50004DC151F14EC152F157C159F158C15AF10E
:102A6000079437EC15F045EC0BF052EF19F066C106
:102A700000F167C101F168C102F169C103F101010F
:102A8000AEEC1FF071EC1DF00401630E826F3BECA5
:102A90000BF004012C0E826F3BEC0BF04FC100F1E8
:102AA00050C101F151C102F152C103F10101AEEC7B
:102AB0001FF071EC1DF00401660E826F3BEC0BF011
:102AC00004012C0E826F3BEC0BF00BEC20F059C193
:102AD00000F15AC101F10101AEEC1FF071EC1DF0E3
:102AE0000401740E826F3BEC0BF0120010820401A3
:102AF000530E826F3BEC0BF004012C0E826F3BEC0B
:102B00000BF083C32AF184C32BF185C32CF186C358
:102B10002DF187C32EF188C32FF189C330F18AC309
:102B200031F18BC332F18CC333F1010159EC20F048
:102B3000D0EC1FF000C166F101C167F102C168F17C
:102B400003C169F18EC32AF18FC32BF190C32CF11D
:102B500091C32DF192C32EF193C32FF194C330F1A1
:102B600095C331F196C332F197C333F1010159ECAA
:102B700020F0D0EC1FF000C14FF101C150F102C1B3
:102B800051F103C152F14CEC20F099C32FF19AC3DB
:102B900030F19BC331F19CC332F19DC333F101018C
:102BA00059EC20F0D0EC1FF000C159F101C15AF1ED
:102BB00037EC15F004012C0E826F3BEC0BF0F0EFBC
:102BC00015F0118E19A002D019AE108C18BE02D0CB
:102BD00018A4108E8251520A02E10F8201D00F9286
:102BE0008251750A02E1108401D010948251550A75
:102BF00002E1108601D0109611A003D011A401D0DB
:102C00001084078410B25EEF16F010A44AEF16F09D
:102C1000B6C166F1B7C167F1B8C168F1B9C169F170
:102C2000BAC16AF1BBC16BF1BCC16CF1BDC16DF140
:102C3000BEC16EF1BFC16FF1C0C170F1C1C171F110
:102C4000C2C172F1C3C173F1C4C174F1C5C175F1E0
:102C5000C6C176F1C7C177F1C8C178F1C9C179F1B0
:102C6000CAC17AF1CBC17BF1CCC17CF1CDC17DF180
:102C7000CEC17EF1CFC17FF1D0C180F1D1C181F150
:102C8000D2C182F1D3C183F1D4C184F1D5C185F120
:102C900052EF16F062C166F163C167F164C168F179
:102CA00065C169F14BC14FF14CC150F14DC151F1BA
:102CB0004EC152F157C159F158C15AF107940FA0B2
:102CC00080EF16F0010192676DEF16F093676DEFDC
:102CD00016F094676DEF16F0956771EF16F080EFC0
:102CE00016F01AEC14F092C104F193C105F194C1ED
:102CF00006F195C107F110EC1FF003BF18EF19F0B2
:102D00001AEC14F00101000E046F000E056F010EA5
:102D1000066F000E076F41EC1FF011A02CD011A21E
:102D20002AD0AEEC1FF0296701D007D004012D0E88
:102D3000826F3BEC0BF016EF19F030C182F4040106
:102D4000300E82273BEC0BF031C182F40401300ECF
:102D500082273BEC0BF032C182F40401300E822753
:102D60003BEC0BF033C182F40401300E82273BECC4
:102D70000BF016EF19F012A8C5D012981AC01BF06C
:102D80001B3A1B42070E1B1600011B50000AD8B449
:102D90004EEF17F000011B50010AD8B4DAEF16F01D
:102DA00000011B50020AD8B4D8EF16F080EF17F0DC
:102DB00080EF17F00BEC20F02AC001F12BC000F1DE
:102DC000D89001330033D890013300330101630EF2
:102DD000046F000E056F000E066F000E076F41ECCA
:102DE0001FF0280E046F000E056F000E066F000E18
:102DF000076F10EC1FF000C12DF00BEC20F028C085
:102E000001F1019F019D29C000F10101A40E046F91
:102E1000000E056F000E066F000E076F41EC1FF0ED
:102E200000C12CF000C104F101C105F102C106F19D
:102E300003C107F1640E006F000E016F000E026FF8
:102E4000000E036F10EC1FF0050E046F000E056FEF
:102E5000000E066F000E076F41EC1FF000C104F179
:102E600001C105F102C106F103C107F10BEC20F02D
:102E70002DC000F110EC1FF000C12EF02EC0E8FFB5
:102E8000050F2D5C03E78A8480EF17F02EC0E8FF62
:102E90000A0F2D5C01E68A9480EF17F000C124F13F
:102EA00001C125F102C126F103C127F10BEC20F08D
:102EB00011EC20F01A501F0BE8CF00F10101640E55
:102EC000046F000E056F000E066F000E076F21ECF9
:102ED0001FF024C104F125C105F126C106F127C167
:102EE00007F110EC1FF003BF02D08A9401D08A844E
:102EF00024C100F125C101F126C102F127C103F16E
:102F000018EF19F000C124F101C125F102C126F129
:102F100003C127F110AE4DD0109E00C108F101C1D0
:102F200009F102C10AF103C10BF1AEEC1FF030C18F
:102F3000D6F131C1D7F132C1D8F133C1D9F108C1CD
:102F400000F109C101F10AC102F10BC103F1010154
:102F50006C0E046F070E056F000E066F000E076FF4
:102F600010EC1FF003BF04D00101550EDA6F1CD026
:102F700008C100F109C101F10AC102F10BC103F15D
:102F80000101A40E046F060E056F000E066F000E01
:102F9000076F10EC1FF003BF04D001017F0EDA6F42
:102FA00003D00101FF0EDA6F1C8E11AE18EF19F07D
:102FB000119E24C100F125C101F126C102F127C1F2
:102FC00003F110A4EBEF17F00401750E826F3BECD8
:102FD0000BF0F0EF17F00401720E826F3BEC0BF078
:102FE00004012C0E826F3BEC0BF0AEEC1FF0296756
:102FF000FFEF17F00401200E826F02EF18F00401BA
:103000002D0E826F3BEC0BF030C182F40401300EC8
:1030100082273BEC0BF031C182F40401300E822791
:103020003BEC0BF004012E0E826F3BEC0BF032C137
:1030300082F40401300E82273BEC0BF033C182F4A2
:103040000401300E82273BEC0BF004016D0E826F01
:103050003BEC0BF004012C0E826F3BEC0BF04FC1EC
:1030600000F150C101F151C102F152C103F101015E
:10307000AEEC1FF071EC1DF00401480E826F3BECCA
:103080000BF004017A0E826F3BEC0BF004012C0E66
:10309000826F3BEC0BF066C100F167C101F168C1C2
:1030A00002F169C103F10101AEEC1FF071EC1DF0FA
:1030B0000401630E826F3BEC0BF004012C0E826F57
:1030C0003BEC0BF066C100F167C101F168C102F190
:1030D00069C103F101010A0E046F000E056F000EB5
:1030E000066F000E076F21EC1FF0000E046F120E2A
:1030F000056F000E066F000E076F41EC1FF0AEEC7F
:103100001FF02AC182F40401300E82273BEC0BF041
:103110002BC182F40401300E82273BEC0BF02CC152
:1031200082F40401300E82273BEC0BF02DC182F4B7
:103130000401300E82273BEC0BF02EC182F4040117
:10314000300E82273BEC0BF02FC182F40401300ECD
:1031500082273BEC0BF030C182F40401300E822751
:103160003BEC0BF004012E0E826F3BEC0BF031C1F7
:1031700082F40401300E82273BEC0BF032C182F462
:103180000401300E82273BEC0BF033C182F40401C2
:10319000300E82273BEC0BF00401730E826F3BEC88
:1031A0000BF004012C0E826F3BEC0BF00BEC20F0CB
:1031B00059C100F15AC101F17CEC1AF00FB2E4EFF1
:1031C00018F00FA016EF19F004012C0E826F3BECE3
:1031D0000BF0200EF86EF76AF66A04010900F5CFCD
:1031E00082F43BEC0BF00900F5CF82F43BEC0BF0E2
:1031F0000900F5CF82F43BEC0BF00900F5CF82F427
:103200003BEC0BF00900F5CF82F43BEC0BF009002E
:10321000F5CF82F43BEC0BF00900F5CF82F43BECE8
:103220000BF00900F5CF82F43BEC0BF045EC0BF012
:103230000F9052EF19F00401630E826F3BEC0BF01C
:1032400004012C0E826F3BEC0BF058EC19F00401DA
:103250002C0E826F3BEC0BF0CBEC19F004012C0E22
:10326000826F3BEC0BF047EC1AF004012C0E826FDE
:103270003BEC0BF00101F80E006FCD0E016F660EF6
:10328000026F030E036F6DEC19F004012C0E826FB8
:103290003BEC0BF05DEC1AF045EC0BF052EF19F043
:1032A00045EC0BF00301C26B0790109261EF1CF02C
:1032B000D8900E0E2FEC09F0E8CF00F10F0E2FEC96
:1032C00009F0E8CF01F1100E2FEC09F0E8CF02F180
:1032D000110E2FEC09F0E8CF03F10101000E046F8D
:1032E000000E056F010E066F000E076F41EC1FF018
:1032F000AEEC1FF02AC182F40401300E82273BECB1
:103300000BF02BC182F40401300E82273BEC0BF052
:103310002CC182F40401300E82273BEC0BF02DC14E
:1033200082F40401300E82273BEC0BF02EC182F4B4
:103330000401300E82273BEC0BF02FC182F4040114
:10334000300E82273BEC0BF030C182F40401300ECA
:1033500082273BEC0BF031C182F40401300E82274E
:103360003BEC0BF004012E0E826F3BEC0BF032C1F4
:1033700082F40401300E82273BEC0BF033C182F45F
:103380000401300E82273BEC0BF004016D0E826FBE
:103390003BEC0BF01200120E2FEC09F0E8CF00F11D
:1033A000130E2FEC09F0E8CF01F1140E2FEC09F009
:1033B000E8CF02F1150E2FEC09F0E8CF03F101017F
:1033C0000A0E046F000E056F000E066F000E076FE9
:1033D00021EC1FF0000E046F120E056F000E066F39
:1033E000000E076F41EC1FF0AEEC1FF02AC182F413
:1033F0000401300E82273BEC0BF02BC182F4040158
:10340000300E82273BEC0BF02CC182F40401300E0D
:1034100082273BEC0BF02DC182F40401300E822791
:103420003BEC0BF02EC182F40401300E82273BEC02
:103430000BF02FC182F40401300E82273BEC0BF01D
:1034400030C182F40401300E82273BEC0BF0040102
:103450002E0E826F3BEC0BF031C182F40401300E72
:1034600082273BEC0BF032C182F40401300E82273C
:103470003BEC0BF033C182F40401300E82273BECAD
:103480000BF00401730E826F3BEC0BF012000A0E7E
:103490002FEC09F0E8CF00F10B0E2FEC09F0E8CF8C
:1034A00001F10C0E2FEC09F0E8CF02F10D0E2FEC1C
:1034B00009F0E8CF03F17CEF1AF0060E2FEC09F0CB
:1034C000E8CF00F1070E2FEC09F0E8CF01F1080E6C
:1034D0002FEC09F0E8CF02F1090E2FEC09F0E8CF4C
:1034E00003F17CEF1AF001010BEC20F0078457C1C7
:1034F00000F158C101F107940101E80E046F800E3C
:10350000056F000E066F000E076F21EC1FF0000E16
:10351000046F040E056F000E066F000E076F41EC7E
:103520001FF0880E046F130E056F000E066F000E5D
:10353000076F10EC1FF00A0E046F000E056F000EEF
:10354000066F000E076F41EC1FF0AEEC1FF001019B
:103550002967B0EF1AF00401200E826FB3EF1AF062
:1035600004012D0E826F3BEC0BF030C182F404019C
:10357000300E82273BEC0BF031C182F40401300E97
:1035800082273BEC0BF032C182F40401300E82271B
:103590003BEC0BF004012E0E826F3BEC0BF033C1C1
:1035A00082F40401300E82273BEC0BF00401430E41
:1035B000826F3BEC0BF0120087C32AF188C32BF11A
:1035C00089C32CF18AC32DF18BC32EF18CC32FF14B
:1035D0008DC330F18EC331F190C332F191C333F119
:1035E0000101296B59EC20F0D0EC1FF00101000E15
:1035F000046F000E056F010E066F000E076F21ECC1
:103600001FF00E0E0C6E00C10BF018EC09F00F0E3F
:103610000C6E01C10BF018EC09F0100E0C6E02C11B
:103620000BF018EC09F0110E0C6E03C10BF018EC46
:1036300009F004017A0E826F3BEC0BF004012C0EB2
:10364000826F3BEC0BF00401350E826F3BEC0BF00C
:1036500004012C0E826F3BEC0BF058EC19F0F0EFEC
:1036600013F087C32AF188C32BF189C32CF18AC3D5
:103670002DF18BC32EF18CC32FF18DC330F18EC38E
:1036800031F190C332F191C333F10101296B59EC4F
:1036900020F0D0EC1FF0880E046F130E056F000EA3
:1036A000066F000E076F15EC1FF0000E046F040E7E
:1036B000056F000E066F000E076F21EC1FF0010171
:1036C000E80E046F800E056F000E066F000E076F88
:1036D00041EC1FF00A0E0C6E00C10BF018EC09F063
:1036E0000B0E0C6E01C10BF018EC09F00C0E0C6EF9
:1036F00002C10BF018EC09F00D0E0C6E03C10BF0BB
:1037000018EC09F004017A0E826F3BEC0BF0040117
:103710002C0E826F3BEC0BF00401360E826F3BECFB
:103720000BF004012C0E826F3BEC0BF047EC1AF00F
:10373000F0EF13F087C32AF188C32BF189C32CF172
:103740008AC32DF18BC32EF18CC32FF18DC330F1C1
:103750008FC331F190C332F191C333F1010159ECC0
:1037600020F0D0EC1FF0000E046F120E056F000E5B
:10377000066F000E076F21EC1FF001010A0E046FA7
:10378000000E056F000E066F000E076F41EC1FF074
:10379000120E0C6E00C10BF018EC09F0130E0C6E3B
:1037A00001C10BF018EC09F0140E0C6E02C10BF005
:1037B00018EC09F0150E0C6E03C10BF018EC09F0B3
:1037C00004017A0E826F3BEC0BF004012C0E826F29
:1037D0003BEC0BF00401370E826F3BEC0BF0040165
:1037E0002C0E826F3BEC0BF0CBEC19F0F0EF13F0EA
:1037F00087C32AF188C32BF189C32CF18AC32DF129
:103800008BC32EF18CC32FF18DC330F18EC331F1F8
:1038100090C332F191C333F10101296B59EC20F0CF
:10382000D0EC1FF0880E046F130E056F000E066FAC
:10383000000E076F15EC1FF0000E046F040E056FED
:10384000000E066F000E076F21EC1FF00101E80E5D
:10385000046F800E056F000E066F000E076F41ECBF
:103860001FF0060E0C6E00C10BF018EC09F0070EED
:103870000C6E01C10BF018EC09F0080E0C6E02C1C1
:103880000BF018EC09F0090E0C6E03C10BF018ECEC
:1038900009F004017A0E826F3BEC0BF004012C0E50
:1038A000826F3BEC0BF00401380E826F3BEC0BF0A7
:1038B00004012C0E826F3BEC0BF05DEC1AF0F0EF84
:1038C00013F081B803D02FB01FEF1DF007A8D9EF78
:1038D0001CF00101800E006F1A0E016F060E026FC0
:1038E000000E036F4BC104F14CC105F14DC106F14F
:1038F0004EC107F110EC1FF003BF1FEF1DF06BEC82
:103900001DF04BC100F14CC101F14DC102F14EC19E
:1039100003F107821DEC1EF018C104F119C105F175
:103920001AC106F11BC107F1F80E006FCD0E016F31
:10393000660E026F030E036F10EC1FF00E0E0C6E7E
:1039400000C10BF018EC09F00F0E0C6E01C10BF06A
:1039500018EC09F0100E0C6E02C10BF018EC09F017
:10396000110E0C6E03C10BF018EC09F00784010175
:103970000BEC20F057C100F158C101F107940A0E79
:103980000C6E00C10BF018EC09F00B0E0C6E01C1AF
:103990000BF018EC09F00C0E0C6E02C10BF018ECD9
:1039A00009F00D0E0C6E03C10BF018EC09F01FEFBF
:1039B0001DF007AA1FEF1DF0078401010BEC20F09A
:1039C00057C100F158C101F10794060E0C6E00C1F9
:1039D0000BF018EC09F0070E0C6E01C10BF018EC9F
:1039E00009F0080E0C6E02C10BF018EC09F0090E7C
:1039F0000C6E03C10BF018EC09F0078462C100F1F2
:103A000063C101F164C102F165C103F10794120EB3
:103A10000C6E00C10BF018EC09F0130E0C6E01C116
:103A20000BF018EC09F0140E0C6E02C10BF018EC40
:103A300009F0150E0C6E03C10BF018EC09F0079895
:103A4000079A0401805181197F0B0DE09EA8FED7D3
:103A500014EE00F081517F0BE126E750812B0F011E
:103A6000AD6E21EF1DF092EF0AF018C100F119C1FF
:103A700001F11AC102F11BC103F1000E046F000E27
:103A8000056F010E066F000E076F41EC1FF029A1B4
:103A900060EF1DF02051D8B460EF1DF018C100F1A7
:103AA00019C101F11AC102F11BC103F1000E046F2B
:103AB000000E056F0A0E066F000E076F41EC1FF037
:103AC00012000101045100130551011306510213A4
:103AD0000751031312000101186B196B1A6B1B6B52
:103AE00012002AC182F40401300E82273BEC0BF055
:103AF0002BC182F40401300E82273BEC0BF02CC169
:103B000082F40401300E82273BEC0BF02DC182F4CD
:103B10000401300E82273BEC0BF02EC182F404012D
:103B2000300E82273BEC0BF02FC182F40401300EE3
:103B300082273BEC0BF030C182F40401300E822767
:103B40003BEC0BF031C182F40401300E82273BECD8
:103B50000BF032C182F40401300E82273BEC0BF0F3
:103B600033C182F40401300E82273BEC0BF01200CB
:103B70002FC182F40401300E82273BEC0BF030C1E0
:103B800082F40401300E82273BEC0BF031C182F449
:103B90000401300E82273BEC0BF032C182F40401A9
:103BA000300E82273BEC0BF033C182F40401300E5F
:103BB00082273BEC0BF01200060E1E6E060E1F6EE7
:103BC000060E206E1E2EE2EF1DF01F2EE2EF1DF0FE
:103BD000202EE2EF1DF08B84020E1E6E020E1F6E71
:103BE000020E206E1E2EF2EF1DF01F2EF2EF1DF0C2
:103BF000202EF2EF1DF08B941200FF0E1F6E1FC0DF
:103C000020F0030E1E6E8B841E2E03EF1EF0030E9B
:103C10001E6E202E03EF1EF08B941FC020F0030EAB
:103C20001E6E1E2E11EF1EF0030E1E6E203E11EFB3
:103C30001EF01F2EFFEF1DF012000101005305E1E1
:103C4000015303E1025301E1002BE0EC1EF00BEC09
:103C500020F03951006F3A51016F420E046F4B0E44
:103C6000056F000E066F000E076F21EC1FF000C1FC
:103C700004F101C105F102C106F103C107F118C148
:103C800000F119C101F11AC102F11BC103F107B220
:103C90004EEF1EF015EC1FF050EF1EF010EC1FF071
:103CA00000C118F101C119F102C11AF103C11BF1E0
:103CB00012000BEC20F059C100F15AC101F1060EBF
:103CC0002FEC09F0E8CF04F1070E2FEC09F0E8CF54
:103CD00005F1080E2FEC09F0E8CF06F1090E2FECE4
:103CE00009F0E8CF07F110EC1FF000C124F101C189
:103CF00025F102C126F103C127F1290E046F000E40
:103D0000056F000E066F000E076F21EC1FF0EE0E20
:103D1000046F430E056F000E066F000E076F15EC63
:103D20001FF024C104F125C105F126C106F127C108
:103D300007F121EC1FF000C11CF101C11DF102C10E
:103D40001EF103C11FF1120E2FEC09F0E8CF04F1B0
:103D5000130E2FEC09F0E8CF05F1140E2FEC09F04B
:103D6000E8CF06F1150E2FEC09F0E8CF07F10D0EA4
:103D7000006F000E016F000E026F000E036F21EC4A
:103D80001FF0180E046F000E056F000E066F000E78
:103D9000076F41EC1FF01CC104F11DC105F11EC1EC
:103DA00006F11FC107F115EC1FF06A0E046F2A0E11
:103DB000056F000E066F000E076F10EC1FF012006B
:103DC000BF0EFA6E200E3A6F396BD890003701376C
:103DD00002370337D8B0F1EF1EF03A2FE6EF1EF0AE
:103DE00039073A070353D8B412000331070B80098F
:103DF0003F6F03390F0B010F396F80EC5FF0406F9D
:103E0000390580EC5FF0405D405F396B3F33D8B0DF
:103E1000392739333FA906EF1FF0405139271200E7
:103E2000010130EC20F0D8B0120001010351071954
:103E3000346FF3EC1FF0D8900751031934AF800FA3
:103E400012000101346B17EC20F0D8A02DEC20F00B
:103E5000D8B0120002EC20F00BEC20F01F0E366FF1
:103E600043EC20F00B35D8B0F3EC1FF0D8A00335AD
:103E7000D8B01200362F30EF1FF034B11AEC20F01A
:103E800012000101346B04510511061107110008DD
:103E9000D8A017EC20F0D8A02DEC20F0D8B012005C
:103EA000086B096B0A6B0B6B43EC20F01F0E366F2F
:103EB00043EC20F007510B5DD8A46BEF1FF00651C7
:103EC0000A5DD8A46BEF1FF00551095DD8A46BEF14
:103ED0001FF00451085DD8A07EEF1FF00451085F69
:103EE0000551D8A0053D095F0651D8A0063D0A5FDF
:103EF0000751D8A0073D0B5FD8900081362F58EFAF
:103F00001FF034B11AEC20F0346B17EC20F0D8908D
:103F100047EC20F007510B5DD8A49BEF1FF0065132
:103F20000A5DD8A49BEF1FF00551095DD8A49BEF53
:103F30001FF00451085DD8A0AAEF1FF0003FAAEFC0
:103F40001FF0013FAAEF1FF0023FAAEF1FF0032B63
:103F5000D8B4120034B11AEC20F012000101346B15
:103F600017EC20F0D8B012004CEC20F0200E366F89
:103F7000003701370237033711EE33F00A0E376F7F
:103F8000E7360A0EE75CD8B0E76EE552372FC0EF90
:103F90001FF0362FB8EF1FF034B12981D8901200EE
:103FA00001010A0E346F200E366F11EE29F03451E4
:103FB000376F0A0ED890E652D8B0E726E732372F8F
:103FC000DBEF1FF00333023301330033362FD5EF1D
:103FD0001FF0E750FF0FD8A00335D8B0120029B169
:103FE0001AEC20F01200045100270551D8B0053D0D
:103FF00001270651D8B0063D02270751D8B0073D2A
:10400000032712000051086F0151096F02510A6F16
:1040100003510B6F12000101006B016B026B036B0C
:1040200012000101046B056B066B076B1200033570
:10403000D8A012000351800B001F011F021F031F95
:10404000003F2AEF20F0013F2AEF20F0023F2AEF45
:1040500020F0032B342B032512000735D8A01200C3
:104060000751800B041F051F061F071F043F40EF69
:1040700020F0053F40EF20F0063F40EF20F0072BF7
:10408000342B072512000037013702370337083772
:1040900009370A370B3712000101296B2A6B2B6B8A
:1040A0002C6B2D6B2E6B2F6B306B316B326B336B3C
:1040B000120001012A510F0B2A6F2B510F0B2B6F8E
:1040C0002C510F0B2C6F2D510F0B2D6F2E510F0BF1
:1040D0002E6F2F510F0B2F6F30510F0B306F31514F
:1040E0000F0B316F32510F0B326F33510F0B336F98
:1040F000120000011650FF0A01E11200390EC86ECD
:10410000800EC76E280EC66E000EC56E1550000AD2
:10411000D8B4B4EF20F01550010AD8B4CDEF20F098
:104120001550020AD8B4E6EF20F01550030AD8B4AF
:10413000FFEF20F01550040AD8B427EF21F01550F6
:10414000050AD8B440EF21F01550060AD8B459EF4B
:1041500021F01550070AD8B472EF21F01550080A63
:10416000D8B48BEF21F012001650000AD8B4AAEF91
:1041700021F01650010AD8B4AEEF21F01650020A11
:10418000D8B4B2EF21F01650030AD8B4B6EF21F03C
:104190001650040AD8B429EF22F01650000AD8B4F9
:1041A000BEEF21F01650010AD8B4C2EF21F016502C
:1041B000020AD8B4C6EF21F01650030AD8B4CAEFE9
:1041C00021F01650040AD8B429EF22F01650000A44
:1041D000D8B4CEEF21F01650010AD8B4D2EF21F0B6
:1041E0001650020AD8B4D6EF21F01650030AD8B4FC
:1041F000DAEF21F01650040AD8B429EF22F0165055
:10420000000AD8B4E7EF21F01650010AD8B4EBEF5A
:1042100021F01650020AD8B4EFEF21F01650030A2D
:10422000D8B403EF22F01650040AD8B407EF22F0F6
:104230001650050AD8B40BEF22F01650060AD8B46F
:104240000FEF22F01650070AD8B412EF22F01650E2
:10425000000AD8B416EF22F01650010AD8B41AEFAB
:1042600022F01650020AD8B41EEF22F01650030AAC
:10427000D8B422EF22F01650040AD8B425EF22F069
:104280001650000AD8B42DEF22F01650010AD8B407
:1042900031EF22F01650020AD8B435EF22F0165052
:1042A000030AD8B439EF22F01650040AD8B429EF23
:1042B00022F01650000AD8B443EF22F01650010A3B
:1042C000D8B447EF22F01650020AD8B44BEF22F0D0
:1042D0001650030AD8B44FEF22F01650040AD8B48F
:1042E00029EF22F01650000AD8B450EF22F01650F1
:1042F000010AD8B454EF22F01650020AD8B458EF8D
:1043000022F01650030AD8B45CEF22F01650040ACB
:10431000D8B429EF22F01650000AD8B45DEF22F08D
:104320001650010AD8B461EF22F01650020AD8B430
:1043300065EF22F01650030AD8B469EF22F0165048
:10434000040AD8B46AEF22F01650050AD8B46DEF0B
:1043500022F012009E96C580162A1200E20EC96E47
:10436000162A1200770EC96E162A1200020EE86E87
:104370008AB4E88AE8CFC9FF162A12009E96C58043
:10438000162A1200E20EC96E162A1200790EC96EA4
:10439000162A1200000EC96E162A12009E96C580BB
:1043A000162A1200E20EC96E162A12007A0EC96E83
:1043B000162A120018BC03D0DAC1E8FF04D0185046
:1043C000E844E8441F09E8CFC9FF162A12009E9668
:1043D000C580162A1200E20EC96E162A120011BA02
:1043E00003D011BC01D003D0050E156E3ED00101E3
:1043F000D667FFEF21F0100EC96E01EF22F0D6C193
:10440000C9FF162A1200D7C1C9FF162A1200D8C147
:10441000C9FF162A1200D9C1C9FF162A1200C58485
:10442000162A1200FF0E166E1D9E12009E96C58063
:10443000162A1200E20EC96E162A1200760EC96EF6
:10444000162A1200C584162A1200FF0E166E1D9E33
:104450001200C584152A166A12009E96C580162A77
:104460001200E20EC96E162A12007B0EC96E162AC1
:10447000120011AA04D0230EC96E162A12001C0EB7
:10448000C96E162A12009E96C580162A1200E20EE8
:10449000C96E162A12007C0EC96E162A1200E9D7C0
:1044A0009E96C580162A1200E20EC96E162A1200C8
:1044B0007D0EC96E162A1200DCD79E96C580162A7C
:1044C0001200E20EC96E162A12007E0EC96E162A5E
:1044D0001200CFD7C584162A1200FF0E166E1D9E3D
:1044E00012001650FF0AD8B42FEF23F0390EC86E11
:1044F000800EC76E280EC66E000EC56E1550000ADF
:10450000D8B48AEF22F01550010AD8B49EEF22F0F9
:104510002FEF23F01650000AD8B4DCEF22F016502B
:10452000010AD8B4E0EF22F01650020AD8B4EAEF3C
:1045300022F01650030AD8B4EDEF22F01650000A0C
:10454000D8B4F3EF22F01650010AD8B4F7EF22F0F6
:104550001650020AD8B401EF23F01650030AD8B45B
:1045600004EF23F01650040AD8B40AEF23F01650D3
:10457000050AD8B40DEF23F01650060AD8B413EF8D
:1045800023F01650070AD8B416EF23F01650080A85
:10459000D8B41CEF23F01650090AD8B41FEF23F04B
:1045A00016500A0AD8B425EF23F016500B0AD8B4D7
:1045B00028EF23F02FEF23F09E96C5802EEF23F0F7
:1045C00017B004D04E0EC96E2EEF23F0500EC96EF8
:1045D0002EEF23F0C5842EEF23F0152AFF0E166E62
:1045E00012802FEF23F09E96C5802EEF23F017B098
:1045F00004D04F0EC96E2EEF23F0510EC96E2EEF70
:1046000023F0C5862EEF23F0C9CF24F0C59AC588C4
:104610002EEF23F0C5862EEF23F0C9CF25F0C59AE3
:10462000C5882EEF23F0C5862EEF23F0C9CF26F0E4
:10463000C59AC5882EEF23F0C5862EEF23F0C9CF8B
:1046400027F0C58AC5882EEF23F0C5842EEF23F00E
:10465000FF0E166E12861D9C2FEF23F0162A1200F5
:1046600012B012D012B213D012B414D012A612008B
:1046700007B01200129624C028F025C029F026C0E9
:104680002AF027C02BF01200129012821200129210
:104690001284120000011650FF0A04E11294166AF7
:0646A00071EC22F0120093
:10BF0000E844F926000C160C2B0C3F0C520C640C68
:10BF1000760C860C960CA50CB30CC10CCF0CDC0C6B
:06BF2000E80CF40C000C1B
:00000001FF
